:020000040000FA
:04000000CB303A289F
:040004000034003490
:08000800A000030EA100831209
:1000100005191128831601178312B2308100B1012E
:100020002C2883160113831203140B190310A80D37
:10003000A90DAA0DAB0DAC0DAC16FF302C02031DA3
:100040002C28FA302B02031D2C2832152A08AF0069
:100050002908AE002808AD008B100B11210E83007B
:06006000A00E200E0900B5
:0C007400203084008001840A80300402E7
:10008000031C3C28DA2183160C3085058701831276
:10009000850187010730990000309A0010308316DF
:1000A0008E008312603083168F0083120030831617
:1000B00091009F008312C830831681008312313073
:1000C0009000003083168C00831210308B00BD1B13
:1000D0006F2885196F286400851D6B28ED22D422B6
:1000E00081018E018F010B118B100B108C018B176E
:1000F000872032199320B40B852803108519031427
:10010000BA0DF0303A0203193C2113237828640019
:100110003310B10A311F9228AC01AB01AA01A90129
:10012000A801B101080032110130B7008B13203053
:10013000370783169B001C141A088312A400103082
:10014000370783169B001C141A088312A300A6000D
:100150000230A6060030370783169B001C141A08CD
:100160008312A200A7000130A7068B17331CBE28FC
:1001700022090339A200A309A409A50924082F0212
:10018000031D362923082E02031D362922082D02BD
:10019000031D362901303702031DD3283E18D3280A
:1001A0003E143F14FC2102303702031DDC28BE1828
:1001B000DC28BE143F14082203303702031DE52853
:1001C0003E19E5283E153F14142204303702031D62
:1001D000EE28BE19EE28BE153F1420220530370246
:1001E000031DF7283E1AF7283E163F142C2206302E
:1001F0003702031D0029BE1A0029BE163F143B22F8
:1002000007303702031D09293E1B09293E173F14F9
:100210004D2208303702031D1229BE1B1229BE17BA
:100220003F14582209303702031D1B295E181B2971
:100230005E143F1463220A303702031D2429DE189E
:100240002429DE143F146E220B303702031D2D29A2
:100250005E192D295E153F1479220C303702031DDB
:100260003629DE193629DE153F148722B70A0D30EC
:1002700037020318080096280130B600B400B50014
:10028000B70085018701B2138720B40B54290310EE
:1002900085190314BA0DF0303A0203197C29B50B05
:1002A00054299630B5008621321D44293211331C61
:1002B0005E292D090339AD00AE09AF092F1C442971
:1002C0002D083002031944292D08B0002E1E4429A0
:1002D0008B1320303707BC002F08BB00C52110301E
:1002E0003707BC002E08BB00C52100303707BC0013
:1002F0002D08BB00C5218B1785018701B70AB60100
:100300000D303702031C4429D42208000130370283
:10031000031998220230370203199D220330370255
:100320000319A222043037020319A722053037022D
:100330000319AC22063037020319B1220730370205
:100340000319B622083037020319BB2209303702DD
:100350000319C0220A3037020319C5220B303702B5
:100360000319CA220C3037020319CF2208003F1CA0
:1003700008003F101030BC003E08BB00C5213030E3
:10038000BC005E08BB00C52108008B133B08831628
:100390001C159A0083123C0883169B0055309D0063
:1003A000AA309D009C1464009C18D3291C11831250
:1003B0008B170800831600309B001C141A08831248
:1003C000BD00831610309B001C141A088312BE0057
:1003D000831630309B001C141A088312DE00FF3095
:1003E000C800CA15CB15CC15CD15CE15CF15D01517
:1003F000D115D215D3150800C130BE05FF30DE057A
:100400000130C405C0000030C200C6005F10080003
:10041000C230BE05FF30DE050230C405C00000302A
:10042000C200C6005F100800C430BE05FF30DE0504
:100430000630C405C0000030C200C6005F100800CE
:10044000C830BE05FF30DE050A30C405C0000030EC
:10045000C200C6005F100800D030BE05FF30DE05C8
:100460003D181030BD181130C405C0000030C20066
:10047000C6005F100800E030BE05FF30DE053D1805
:100480001830BD181930C405C0001830C200C600AD
:100490005F105F17C411441208007F30BE05C030E2
:1004A000DE050830C505C1000030C300C7000800E4
:1004B000BF30BE05C030DE051030C505C1000030BC
:1004C000C300C70008003F30BE05C130DE05303034
:1004D000C505C1000030C300C70008003F30BE059D
:1004E000C230DE055030C505C1000030C300C70072
:1004F00008003F30BE05C430DE053D188030BD1811
:100500008830C505C1000030C300C70008003F3077
:10051000BE05C830DE053D18C030BD18C830C50561
:10052000C100C030C300C700DF174513C513080062
:100530001030850600308706080020308506003020
:100540008706080021308506003087060800223023
:1005500085060030870608000030850602308706D1
:100560000800023085060230870608000030850644
:100570000430870608000030850601308706080031
:1005800000308506213087060800003085061130CE
:10059000870608000030850608308706080000300E
:1005A00085061830870608003E18FC21BE18082270
:1005B0003E191422BE1920223E1A2C22BE1A3B22BA
:1005C0003E1B4D22BE1B58225E186322DE186E228F
:1005D0005E197922DE1987220800B601B401B5013F
:1005E0003D1CF52ABD01BD14F72ABD013D143D088F
:1005F000B6006400FB2AFC2AFD2AFE2AFF2AFF30EF
:10060000B51B8500B51F8501B40BF92AB50BF92A76
:100610000310B60CB608031DF92A0030BC003D08D3
:10062000BB00C52108008F08031908008F0178302E
:100630008E00C80F3D2DC80A441C432B461C342B8A
:10064000CA1C252BCA014A15512B4A1D2A2BCA0147
:10065000CA15512BCA1D2F2BCA014A16512B4A1EEF
:10066000512BCA01CA14512B4A1D392BCA014A16F3
:10067000512BCA1D3E2BCA014A16512B4A1E512B23
:10068000CA01CA14512BCA1C482BCA014A15512B46
:100690004A1D4D2BCA01CA15512B4A1E512BCA01A6
:1006A0004A15C41C782BC61C692BCB1C5A2BCB01BA
:1006B0004B15862B4B1D5F2BCB01CB15862BCB1DF2
:1006C000642BCB014B16862B4B1E862BCB01CB14F8
:1006D000862B4B1D6E2BCB014B16862BCB1D732B04
:1006E000CB014B16862B4B1E862BCB01CB14862BB6
:1006F000CB1C7D2BCB014B15862B4B1D822BCB01AD
:10070000CB15862B4B1E862BCB014B15441DAD2BD9
:10071000461D9E2BCC1C8F2BCC014C15BB2B4C1D8E
:10072000942BCC01CC15BB2BCC1D992BCC014C169A
:10073000BB2B4C1EBB2BCC01CC14BB2B4C1DA32BB9
:10074000CC014C16BB2BCC1DA82BCC014C16BB2BC3
:100750004C1EBB2BCC01CC14BB2BCC1CB22BCC0124
:100760004C15BB2B4C1DB72BCC01CC15BB2B4C1EF9
:10077000BB2BCC014C15C41DE32BC61DD42BCD1CAB
:10078000C52BCD014D155F13F12B4D1DCA2BCD018E
:10079000CD15F12BCD1DCF2BCD014D16F12B4D1EBF
:1007A000F12BCD01CD14F12B4D1DD92BCD014D16C3
:1007B000F12BCD1DDE2BCD014D16F12B4D1EF12B56
:1007C000CD01CD14F12BCD1CE82BCD014D15F12B16
:1007D0004D1DED2BCD01CD15F12B4D1EF12BCD0176
:1007E0004D155F1B1A2C441E1A2C461E0B2CCE1CBA
:1007F000FC2BCE014E15282C4E1D012CCE01CE1502
:10080000282CCE1D062CCE014E16282C4E1E282C30
:10081000CE01CE14282C4E1D102CCE014E16282CA5
:10082000CE1D152CCE014E16282C4E1E282CCE0186
:10083000CE14282CCE1C1F2CCE014E15282C4E1D5C
:10084000242CCE01CE15282C4E1E282CCE014E1560
:10085000C51D4F2CC71D402CCF1C312CCF014F156F
:100860005D2C4F1D362CCF01CF155D2CCF1D3B2CA1
:10087000CF014F165D2C4F1E5D2CCF01CF145D2C88
:100880004F1D452CCF014F165D2CCF1D4A2CCF019B
:100890004F165D2C4F1E5D2CCF01CF145D2CCF1C4D
:1008A000542CCF014F155D2C4F1D592CCF01CF1566
:1008B0005D2C4F1E5D2CCF014F15451E842C471E0D
:1008C000752CD01C662CD0015015922C501D6B2C11
:1008D000D001D015922CD01D702CD0015016922C26
:1008E000501E922CD001D014922C501D7A2CD00185
:1008F0005016922CD01D7F2CD0015016922C501ED9
:10090000922CD001D014922CD01C892CD0015015DF
:10091000922C501D8E2CD001D015922C501E922C52
:10092000D0015015C51EB92CC71EAA2CD11C9B2C5A
:10093000D1015115C72C511DA02CD101D115C72CA7
:10094000D11DA52CD1015116C72C511EC72CD10188
:10095000D114C72C511DAF2CD1015116C72CD11D5C
:10096000B42CD1015116C72C511EC72CD101D11462
:10097000C72CD11CBE2CD1015115C72C511DC32C25
:10098000D101D115C72C511EC72CD1015115451FBE
:10099000EF2C471FE02CD21CD12CD2015215DF13B3
:1009A000FD2C521DD62CD201D215FD2CD21DDB2CD4
:1009B000D2015216FD2C521EFD2CD201D214FD2C58
:1009C000521DE52CD2015216FD2CD21DEA2CD2016B
:1009D0005216FD2C521EFD2CD201D214FD2CD21C1D
:1009E000F42CD2015215FD2C521DF92CD201D21536
:1009F000FD2C521EFD2CD2015215DF1B262DC51FCA
:100A0000262DC71F172DD31C082DD3015315342DA8
:100A1000531D0D2DD301D315342DD31D122DD3010C
:100A20005316342D531E342DD301D314342D531D9E
:100A30001C2DD3015316342DD31D212DD301531654
:100A4000342D531E342DD301D314342DD31C2B2D10
:100A5000D3015315342D531D302DD301D315342D0F
:100A6000531E342DD3015315B7214008C40041084B
:100A7000C5005F18DF145F1CDF104808C9000C3088
:100A80004A05031D05120C304B05031D85120C3061
:100A90004C05031D05100C304D05031D85100C3051
:100AA0004E05031D87100C304F05031D07110C3038
:100AB0005005031D07100C305105031D87120C3023
:100AC0005205031D07120C305305031D87114908F9
:100AD0000E020318972D12304A05031D0516123019
:100AE0004B05031D851612304C05031D05141230ED
:100AF0004D05031D851412304E05031D8714123059
:100B00004F05031D071512305005031D0714123041
:100B10005105031D871612305205031D07161230AA
:100B20005305031D8715FF304802031908008F087D
:100B3000031D0800872049080E02031C972D18305A
:100B40004A05031D051206304A05031D0516183017
:100B50004B05031D851206304B05031D8516183005
:100B60004C05031D051006304C05031D05141830F7
:100B70004D05031D851006304D05031D85141830E5
:100B80004E05031D871006304E05031D87141830CF
:100B90004F05031D071106304F05031D07151830BB
:100BA0005005031D071006305005031D07141830AB
:100BB0005105031D871206305105031D8716183095
:100BC0005205031D071206305205031D0716183083
:100BD0005305031D871106305305031D87150800B3
:084000000300030006000900A3
:02400E00CC33B1
:10420000010078007A007C007E007B0079007F004E
:104210007D007A0078007E007C007D007F007900C0
:104220000200F200F600FA00FE00F200F600FA00CA
:10423000FE00F200F600FA00FE00F200F600FA00BE
:10424000FF00050005000500050009000900090040
:1042500009000D000D000D000D00110011001100EE
:104260000100FF00FF00FF00FF00FF00FF00FF0054
:10427000FF00FF00FF00FF00FF00FF00FF00FF0046
:10428000FF007B00FF00FF00FF00FF00FF00FF00BA
:10429000FF00FF00FF00FF00FF00FF00FF00FF0026
:1042A000FF00FE00FF00FF00FF00FF00FF00FF0017
:1042B000FF00FF00FF00FF00FF00FF00FF00FF0006
:1042C000FF001100FF00FF00FF00FF00FF00FF00E4
:1042D000FF00FF00FF00FF00FF00FF00FF00FF00E6
:1042E000FF00FF00FF00FF00FF00FF00FF00FF00D6
:1042F000FF00FF00FF00FF00FF00FF00FF00DD00E8
:00000001FF
